:100000000C0C0600720073000604260486058F0996
:100010008F0906058F0906048F098F098F098F093B
:100020008F098F098F098F098F098F098F098F0910
:100030008F098F098F098F098F098F098F098F0900
:100040008F098F098F098F098F098F098F098F09F0
:100050008F098F098F098F098F098F098F098F09E0
:100060008F098F098F098F098F098F098F098F09D0
:100070008F098F098F098F098F098F098F098F09C0
:100080008F098F098F098F098F098F098F098F09B0
:100090008F098F098F098F098F098F098F098F09A0
:1000A0008F098F098F098F098F098F098F098F0990
:1000B0008F098F098F098F098F0986048F098F098E
:1000C0008F098F098F098F098F0906058F0926056A
:1000D00006048F0926048F0966066F0A6C0A8F09C9
:1000E0008F098F098F098F098F098F098F092605BD
:1000F0008F0926048F0946067E0A7B0A2605840995
:1001000026048F098F097B0AFA0C32006E0C33002B
:1001100000000000F302880AF202860A0008FA0CC6
:100120003200FA0C330000000000F302930AF202DE
:04013000910A000828
:021FFE000A00D7
:00000001FF
